:020000040000FA
:100000007E007B007A00580906056D095A070C0A24
:10001000BA025A060C0A6600FE06100ABE02150A4B
:10002000DE06140ABE02150A66005F09620962094B
:10003000000000000000C606520A6500620962095D
:1000400000000000000000000000000000000000B0
:1000500000000000000000000000000000000000A0
:10006000000000000000000000000000C607520A67
:100070000400BB02FB07150A840C3A007B00FE0655
:10008000050A3F0766043F066605860562096209A0
:10009000C6064C090605050A6F060008AF026F0682
:1000A0007F0200086500FA0706047E006F00050A5B
:1000B00065006600FC0C0500E60C06000008FF0C5D
:1000C00025000008030C3D00020C3C00FD02690AFB
:1000D00000083C00FC026A0A660A020C2E00050CAD
:1000E0002D00B90C2C00EC02730AED02730AEE022B
:1000F000730A0008000A000A000A000A000A000A3F
:10010000000A000A000A000A000A000A000A000A9F
:10011000000A000A000A000A000A000A000A000A8F
:10012000000A000A000A000A000A000A000A000A7F
:10013000000A000A000A000A000A000A000A000A6F
:021FFE00FD0FD5
:00000001FF
